:04000000B601DE293E
:100008000800B616B61EB612B6190E28B615472041
:10001800031835280830A3005B20A20DA30B102875
:10002800B61E402065206120B61A35203A202208E5
:100038000310D929B616B61EB61236192828FE3965
:10004800B70036150310D929361A3028A6003616F7
:1000580047200318352826084E2003183528B61ED1
:10006800D9294020652036113612B6113A08840085
:1000780038088417800446283A088400380980051F
:100088008417800508003A20652040206120370841
:10009800B6190138A2000830A300A20D03183A20AF
:1000A800031C402065206120A30B51283A206520BD
:1000B8003A08840038080005FF3E3B0884003909E7
:1000C80043283B08840039083D2864007F20031832
:1000D8006928CE20A8010830A300CF207F2003186C
:1000E800A80AAB1EA801A20CA30B7128AB1AA21375
:1000F800CF20220808003A088400380884178004B2
:10010800841300052B1B3806FF3E0800A4002908AD
:100118000319D929D421A00025188317240884009D
:10012800200880008313A40AA9038B280408A600CA
:100138003A0884008030B7050830A7000310031878
:10014800B70AB420A60CA70BA3280000AB1A370CDB
:10015800B420DC210314B4202F08A3002E083C2966
:100168008413AB1FC328000838042B1F38068000EF
:10017800841700083804031C38068000CF280008BC
:100188003804031C38062B1B3806800084173809EE
:100198008005CF2837172B081F39003EA1002A08F1
:1001A8000E3E0318A10A371F49293713A000023051
:1001B8007C214929B71329080319B7170430A80067
:1001C800250EEB202508EB20240EEB2024080F3900
:1001D800F63E0318073E0A3EF128A000A8030319BB
:1001E800B71329080319FB28280203180800200858
:1001F800031DB713B71B0800303ED42901308A000D
:1002080028080739820701340234043408341034CA
:1002180020344034803483178001840AFF3E031D54
:100228001029D929210820040319A00A8030201A8E
:10023800A1062019A106A018A106210DA00DA10D47
:10024800D92903178D0083168C130C1483120C08FC
:10025800D92903178C0083168C130C1555308D0083
:10026800AA308D008C148C1837290C11D929A301B8
:10027800A200FF30A207031CA307031CD9290330DF
:10028800A100E63049213D29A101FC3EA000A109B9
:10029800031C5429FF300000A00703184F29A007AA
:1002A8006400A10F4E290800A8000221A001A101A5
:1002B800A81DA000A819A1002008D929A201A301FE
:1002C8006929A10CA00CA20DA30DFF3E03186529F6
:1002D8002308A1002208A000D9290310A00DA10D10
:1002E800FF3E031871292008D9290310A10CA00C7E
:1002F800FF3E031879292008D929A101A301A200EA
:1003080002309229A301A20003309229A301A2007E
:1003180001309229A301A20006309229A8002308DF
:100328002102031D992922082002043003180130F4
:10033800031902302805031DFF30D929A501A4019E
:100348001030A600210DA40DA50D2208A402230833
:10035800031C230FA5020318B8292208A4072308A1
:100368000318230FA5070310A00DA10DA60BA6299E
:100378002008D9291030A800A101A001A70CA60CBB
:10038800031CCC292208A00723080318230FA10760
:10039800A10CA00CA50CA40CA80BC2292408D929CF
:1003A800840031088A003008820083130313831203
:1003B800640008002030840060308A011021A030D9
:1003C800840050308A0110211030840060308A0186
:1003D8000F219030840060308A010F218316D601E6
:1003E800D50120308400603083128A011021A030AA
:1003F800840050308A0110211030840060308A0156
:100408000F219030840060308A010F218316073055
:100418009F00990183129801831602309800DF012A
:10042800E00186100611880107108710071188015E
:100438000710871007118712890183128712831604
:1004480087128312071001308A013B210714643098
:100458008A013B218A150A12342B091183163408A4
:10046800831288008A110A123E2A09158316360853
:100478008312880007110000071509110800831668
:100488004330B60083128A0139228316FF30880070
:10049800831209158710000008088316C400831208
:1004A8008714091183168801831208008316013006
:1004B800C50083128A110A12BC22831626088312E9
:1004C800A000831627088312A1000830A200A30108
:1004D8008A01A2212408B2002508B30032088A0143
:1004E8005821B2002108B3003208A0003308A10047
:1004F80008308A0162218316C10083128A014322CF
:10050800640083164508003C8A110A128312031DF1
:10051800952A831644084104C30083128A110A12DB
:100528009A2A831644084106C3008312831646306C
:10053800B60083128A01392283162008B400831278
:100548008A0131227D088316B40083128A01312280
:1005580083164230B60083128A0139228316430873
:10056800B40083128A0131228316C5018312080060
:10057800831628088312A600831629088312A70069
:100588002030A200A3018A01BE218316AE00831287
:1005980025088316AF0026088312A00083162708B3
:1005A8008312A1000830A200A3018A01A2218316A8
:1005B800AC00831221088316AD002E082C07831285
:1005C800B20083162F080318013E2D078312B300CB
:1005D80000303207FB0010300318013E3307FC00DF
:1005E8007C08FD00FE017B088316A000A1014630AF
:1005F800B60083128A01392283162008B4008312B8
:100608008A0131227D088316B40083128A013122BF
:10061800080083164E084B07A600A701A70D4F0830
:100628004C07A800A901A90D83128A015E2283162E
:100638004E084B02A600A701031CA7034F084C074E
:10064800A800A901A90D83128A015E2283164B080E
:100658004E07A600A701A70D4F084C02A800A90144
:10066800031CA90383128A015E2283164E084B02DB
:10067800A600A701031CA7034F084C02A800A90164
:10068800031CA90383128A015E2283164F084B07B5
:10069800A600A701A70D4E084C07A800A901A90D9F
:1006A80083128A015E2283164F084B02A600A70117
:1006B800031CA7034C084E07A800A901A90D831223
:1006C8008A015E2283164B084F07A600A701A70DD3
:1006D8004E084C02A800A901031CA90383128A0131
:1006E8005E2283164F084B02A600A701031CA7032E
:1006F8004E084C02A800A901031CA90383128A0111
:100708005E2208008316CE014D08CF008312023006
:10071800A600A70183164D088312A200A3018A012F
:10072800BE21B2002508B3003208023C8316AA0095
:1007380083123308031C013E003C8316AB0083126E
:10074800640083164E084F028A110A128312031C92
:10075800FF2B8A010D2364008A110A128316831065
:10076800AB1F831483128318D72B0430A600A7016C
:1007780083164E088312A200A3018A01BE21B2008B
:100788002508B3000630B2070318B30A32088316E7
:10079800AA07831233080318013E8316AB07831296
:1007A8008A110A12FA2B83164F084E028312B200DE
:1007B800B301031CB3030430A600A7013208A2004A
:1007C8003308A3008A01BE21B2002508B3000A300D
:1007D800B2070318B30A32088316AA07831233082C
:1007E8000318013E8316AB07CF0383128316CE0A84
:1007F80083128A01A42B08008316CE014D08CF006E
:1008080083120230A600A70183164D088312A200A6
:10081800A3018A01BE21B2002508B3003208023CB8
:100828008316AA0083123308031C013E003C83167A
:10083800AB008312640083164E084F028A110A1215
:100848008312031C472C8A010D230430A600A7013C
:1008580083164E088312A200A3018A01BE21B200AA
:100868002508B3000630B2070318B30A3208831606
:10087800AA07831233080318013E8316AB07CE0A72
:1008880083128A011E2C08008316CE014D08CF0062
:1008980083120230A600A70183164D088312A20016
:1008A800A3018A01BE21B2002508B3003208023C28
:1008B8008316AA0083123308031C013E003C8316EA
:1008C800AB008312640083164E084F028A110A1285
:1008D8008312031C982C8A010D2383164F084E029D
:1008E8008312B200B301031CB3030430A600A701AE
:1008F8003208A2003308A3008A01BE21B2002508ED
:10090800B3000A30B2070318B30A32088316AA07DD
:10091800831233080318013E8316AB070330CF0256
:10092800CE0A83128A01662C08008316CE014D0870
:10093800CF0083120230A600A70183164D08831248
:10094800A200A3018A01BE21B2002508B300320823
:10095800023C8316AA0083123308031C013E003CA4
:100968008316AB008312640083164E084F028A1167
:100978000A128312031CE82C8A010D2383164F08E0
:100988004E028312B200B301031CB3030430A60065
:10099800A7013208A2003308A3008A01BE21B200D1
:1009A8002508B3000A30B2070318B30A32088316C1
:1009B800AA07831233080318013E8316AB07CF0337
:1009C800CE0A83128A01B72C08008A110A1221253F
:1009D80083164608BA008312640083163A08470251
:1009E8008A110A128312031C202D83164908BD00A0
:1009F8008312640083163D084A028A110A12831280
:100A0800031C182D83163A08A600A7013D08A80064
:100A1800A90183128A015E2283165A08BD078A112A
:100A28000A128312031CFD2C83165A08BA078A116E
:100A38000A128312031CF02C08006400831646086F
:100A480047028A110A1283120318302D83164608AA
:100A58004702C607C70283126400831649084A0280
:100A68008A110A12831203183F2D831649084A0275
:100A7800C907CA028312080083165C08A600A701EA
:100A88005E08A800A9018312831628088312A00013
:100A9800831629088312A10083165D0883128A0130
:100AA8008A218A110A12031D642D8A015E22831687
:100AB800A80A0319A90A8A110A128312031D482DCC
:100AC800013083165C07A600A701A70D5E08A800E1
:100AD800A9018312831628088312A0008316290807
:100AE8008312A10083165D0883128A018A218A1164
:100AF8000A12031D902D8A015E2283165A08A80740
:100B08008A110A128312031C6E2D8316A80A8A11F1
:100B18000A128312031D6E2D080083165E08A800B2
:100B2800A9015C08A600A701831283162608831270
:100B3800A000831627088312A10083165B0883127E
:100B48008A018A218A110A12031DB52D8A015E22A3
:100B58008316A60A0319A70A8A110A128312031D0B
:100B6800992DFF3083165E07A800FF300318013E59
:100B7800A9005C08A600A701831283162608831221
:100B8800A000831627088312A10083165B0883122E
:100B98008A018A218A110A12031DE32D8A015E2225
:100BA80083165A08A6078A110A128312031CC12D3C
:100BB8008316A60A8A110A128312031DC12D080082
:100BC8008A012125831646084702BF0049084A02C0
:100BD800C000640040083F028A110A128312031CF5
:100BE800732E831640088312A000A10102308A01E7
:100BF8007421B2002108B30083163F088312320221
:100C08008316AA0083123308031CFF3E8316AB0029
:100C18004908A800A9014608A600A701831283165F
:100C280026088312A000831627088312A1008316C2
:100C3800470883128A018A218A110A12031D722E1B
:100C480064008A110A1283168310AB1F831483125F
:100C58008318462E831640088312A000A101023093
:100C68008A017421B2002108B30032088316AA074A
:100C7800831233080318013E8316AB0783128A11C7
:100C88000A12672E83163F0840028312B200B3018E
:100C9800031CB3030230A600A7013208A2003308E0
:100CA800A3008A01BE21B2002508B30032088316CA
:100CB800AA07831233080318013E8316AB07A80A54
:100CC8000319A90A83128A015E228316A60A031948
:100CD800A70A8A110A128312031D132E080083160D
:100CE8003F088312A000A10102308A017421B200DA
:100CF8002108B30083164008831232028316AA0023
:100D080083123308031CFF3E8316AB004608A60077
:100D1800A7014908A800A90183128316280883128D
:100D2800A000831629088312A10083164A0883129B
:100D38008A018A218A110A12031DF02E64008A1181
:100D48000A1283168310AB1F831483128318C42ED0
:100D580083163F088312A000A10102308A01742182
:100D6800B2002108B30032088316AA078312330899
:100D78000318013E8316AB0783128A110A12E52E67
:100D8800831640083F028312B200B301031CB30369
:100D98000230A600A7013208A2003308A3008A0186
:100DA800BE21B2002508B30032088316AA078312B1
:100DB80033080318013E8316AB07A60A0319A70ACE
:100DC80083128A015E228316A80A0319A90A8A11C6
:100DD8000A128312031D912E08008A012125831609
:100DE8004608BA008312640083163A0847028A113B
:100DF8000A128312031C192F83163A08A600A701AA
:100E08004908A800A90183128A015E2283164A08AC
:100E1800A800A90183128A015E2283165A08BA071C
:100E28008A110A128312031CF72E83164908BA0086
:100E38008312640083163A084A028A110A1283123E
:100E4800031C3F2F83163A08A800A9014608A600EC
:100E5800A70183128A015E2283164708A600A7010C
:100E680083128A015E2283165A08BA078A110A1267
:100E78008312031C1D2F080083164630B600831208
:100E88008A0139228316B40183128A01312283161A
:100E98001030B40083128A01312283164C30B60018
:100EA80083128A01392283164230B60083128A01DE
:100EB800392283160130BA00831264008130831608
:100EC8003A028A110A12831203188A2F83160130F4
:100ED800BD0083126400213083163D028A110A1274
:100EE80083120318832F8316B40183128A013122D7
:100EF8008316BD0A8A110A128312031D6E2F8316E8
:100F0800BA0A8A110A128312031D612F0800831678
:100F18004630B60083128A0139228316B40183123F
:100F28008A01312283161030B40083128A013122DB
:100F3800080083164630B60083128A0139228316C8
:100F4800B40183128A0131228316B40183128A0103
:100F5800312283164C30B60083128A013922831657
:100F68004230B60083128A01392283160130BA0052
:100F780083126400113083163A028A110A1283120E
:100F88000318E72F83160130BD0083126400213057
:100F980083163D028A110A1283120318E02F831662
:100FA8002030B40083128A0131228316BD0A8A11C7
:100FB8000A128312031DCA2F8316BA0A8A110A124B
:100FC8008312031DBD2F080083164630B600831216
:100FD8008A0139228316B40183128A0131228316C9
:100FE800B401831208008A0140278A018B278A01ED
:100FF8009D278A01E827080083164030B60083122F
:101008008A0139228316BA018312640008308316D4
:101018003A028A150A12831203183A2883163A08E4
:10102800073C8A150A128312031C31288A150A12F2
:1010380023208316B40083128A150A123128083037
:101048008A0083163A0883128207303487340734BB
:101058001F3452347F34203400348A0131228316FD
:10106800BA0A8A150A128312031D09288316443006
:10107800B60083128A0139228316BA0183126400EA
:10108800063083163A028A150A1283120318722848
:1010980083163A08053C8A150A128312031C69282C
:1010A8008A150A125D208316B40083128A150A1263
:1010B800692808308A0083163A08831282070034A8
:1010C80000347F34003410347F348A01312283168F
:1010D800BA0A8A150A128312031D432883165A3046
:1010E800B60083128A0139228316B40183128A0159
:1010F800312283165B30B60083128A0139228316A7
:101108000130B40083128A01312283165830B600A8
:1011180083128A01392283161630B40083128A0199
:1011280031228A0140278A019D2783164630B6005E
:1011380083128A0139228316B40183128A0131226B
:101148008316B40183128A01312283164C30B6000B
:1011580083128A01392283164230B40083128A012D
:1011680031228316B40183128A01312283165D303D
:10117800B60083128A01392283160430B400831220
:101188008A01312283168630B40083128A01312203
:1011980083165930B60083128A0139228316143017
:1011A800B40083128A01312283164C30B6008312B0
:1011B8008A013922080083164630B60083128A0154
:1011C80039227B088316B40083128A0131227C08F5
:1011D8008316B40083128A01312283163708B600B9
:1011E80083128A013922080083163A085C3E84007B
:1011F80000088312B200FF30A200A20A22080F3CA6
:101208008A150A12031C2B298A150A121721320281
:101218008A150A12031D012922088316D200831297
:101228008A150A122B2909308A00220882073034CD
:101238003134323433343434353436343734383462
:101248003934613462346334643465346634080094
:101258002030A600A701831628088312A20083164F
:1012680029088312A3008A01BE21B2002508B30011
:101278003208A0003308A1000830A200A3018A01A7
:10128800A221B2002108B300831626088312A00009
:10129800831627088312A1000830A200A3018A013F
:1012A800A221B4002108B50032083407FB00330836
:1012B8000318013E3507FC008A150A1291292030CF
:1012C800A600A701831628088312A20083162908FE
:1012D8008312A3008A01BE21B2002508B300831639
:1012E80026088312A000831627088312A10008305D
:1012F800A200A3018A01A221B4002108B500320886
:10130800B40733080318013EB50700303407FB0063
:1013180010300318013E3507FC008A150A12DF2039
:1013280083164230B60083128A01392283163508A3
:10133800B40083128A01312208000730BA00403015
:10134800B8002030AA00AB01AE01AF010230A900FD
:10135800831635088312A400A5019A30B000B101A4
:101368008A01DE2008000730BA008030B80020303B
:10137800AA00AB018A0169205D3C8A150A12031D87
:10138800BE290230A9006930B000B101A5015C3066
:101398008A018A208316BA018312640002308316F8
:1013A8003A028A150A1283120318E9298A150A12C1
:1013B800F82083163A085C3E840052088000BA0A76
:1013C8008A150A128312031DD1295C08A000A10105
:1013D80004308A017421B2002108B3005D08320488
:1013E800FF0008000730BA008030B8002030AA009B
:1013F800AB018A0169205D3C8A150A12031DFD298B
:101408000430A9006930B000B101A5015C308A013F
:101418008A208316BA0183126400043083163A02C4
:101428008A150A1283120318282A8A150A12F82024
:1014380083163A085C3E840052088000BA0A8A156E
:101448000A128312031D102A5C08A000A1010430AF
:101458008A017421B2002108B3005D083204FF003C
:101468005E08A000A10104308A017421B20021089D
:10147800B3005F0832048316B000831208000730F7
:10148800BA008030B8002030AA00AB018A01692078
:101498005D3C8A150A12031D4A2A0630A9006930E4
:1014A800B000B101A5015C308A018A208316BA0117
:1014B80083126400063083163A028A150A128312D0
:1014C8000318752A8A150A12F82083163A085C3E12
:1014D800840052088000BA0A8A150A128312031D72
:1014E8005D2A5C08A000A10104308A017421B200C1
:1014F8002108B3005D083204FF005E08A000A101C6
:1015080004308A017421B2002108B3005F08320454
:101518008316B00083126008A000A10104308A017C
:101528007421B2002108B300610832048316B100A7
:10153800831208000730BA008030B8002030AA00B3
:10154800AB018A0169205D3C8A150A12031DA52A90
:101558008A0169208316D20030305202DA0052081C
:10156800B500831208000730BA008030B800203078
:10157800AA00AB018A0169205D3C8A150A12031D85
:10158800BE2A0830A9006930B000B101A5015C305D
:101598008A018A208316BA018312640008308316F0
:1015A8003A028A150A1283120318E92A8A150A12BE
:1015B800F82083163A085C3E840052088000BA0A74
:1015C8008A150A128312031DD12A5C08A000A10102
:1015D80004308A017421B2002108B3005D08320486
:1015E8008316C60083125E08A000A10104308A0198
:1015F8007421B2002108B3005F0832048316C700C3
:1016080083126008A000A10104308A017421B2008D
:101618002108B300610832048316C90083126208E6
:10162800A000A10104308A017421B2002108B3008E
:10163800630832048316CA00831208007F088316E1
:10164800CB003008CC003108CD00831208007F0899
:101658008316A600A7013008A800A9018312080074
:101668008A150A1200208A01F727C530FB00FC0101
:1016780083164C30B70083128A150A12DF208316AE
:101688004230B60083128A0139228316BA018312C6
:101698006400163083163A028A150A128312031858
:1016A8008B2B83163A08153C8A150A128312031CE1
:1016B800822B8A150A1266238316B40083128A15B0
:1016C8000A12822B0B308A0083163A08831282078B
:1016D800503449344334203443346F346E347434D2
:1016E80072346F346C346C3465346434203453345D
:1016F8004534443431343334333430348A0131227C
:101708008316BA0A8A150A128312031D4C2BE3307A
:10171800FB00FC0183164C30B70083128A150A12AD
:10172800DF2083164230B60083128A0139228316DD
:10173800BA01831264001B3083163A028A150A1212
:1017480083120318E22B83163A081A3C8A150A12E8
:101758008312031CD92B8A150A12B8238316B400E6
:1017680083128A150A12D92B0B308A0083163A087D
:10177800831282075534733469346E3467342034E5
:1017880050346934633442346134733469346334B3
:10179800503472346F3420345634653472342E34F5
:1017A800203432342E34343432348A0131228316D0
:1017B800BA0A8A150A128312031D9E2B0530FB00F4
:1017C8000130FC0083164C30B70083128A150A12C8
:1017D800DF2083164230B60083128A01392283162D
:1017E800BA0183126400153083163A028A150A1268
:1017F80083120318342C83163A08143C8A150A12EB
:101808008312031C2B2C8A150A1210248316B40089
:1018180083128A150A122B2C0C308A0083163A0878
:1018280083128207523461346E346A3469347434F2
:101838002034443469346F346C3420342D342034EB
:1018480043344F344D3450345334793473348A012B
:1018580031228316BA0A8A150A128312031DF62B3F
:101868002430FB000130FC0083164C30B700831293
:101878008A150A12DF2083164230B60083128A01C5
:1018880039228316BA0183126400173083163A028C
:101898008A150A1283120318882C83163A08163CF4
:1018A8008A150A128312031C7F2C8A150A126224D5
:1018B8008316B40083128A150A127F2C0C308A0012
:1018C80083163A0883128207683474347434703487
:1018D8003A342F342F347734773477342E346334D2
:1018E8006F346D34703473347934733431342E3446
:1018F80063346F346D348A0131228316BA0A8A152B
:101908000A128312031D482C8316C601C901FF3031
:10191800C7007F30CA000130DA0083128A01F1263D
:1019280083160430C6000430C900FB30C7007B3082
:10193800CA0083128A01F1260F30A300A0308A0161
:101948003C218A01F7270530FB00FC0183164C3047
:10195800B70083128A150A12DF2083164230B600B8
:1019680083128A0139228316BA0183126400143063
:1019780083163A028A150A1283120318F72C831663
:101988003A08133C8A150A128312031CEE2C8A1596
:101998000A12D4248316B40083128A150A12EE2C74
:1019A8000C308A0083163A08831282074434523472
:1019B8004134573420344734523441345034483455
:1019C8004934433420344434453453344934473457
:1019D8004E3453348A0131228316BA0A8A150A1200
:1019E8008312031DBA2C83162330CB004030CC0061
:1019F8000A30CD00831264001F3083164D028A1509
:101A08000A1283120318122D8A0186230A308316BC
:101A1800CD078A150A128312031CFF2C8316643023
:101A2800CB004030CC000A30CD00831264001F3058
:101A380083164D028A150A12831203182D2D8A0166
:101A480000240A308316CD078A150A128312031C54
:101A58001A2D8316A030CB004030CC000A30CD00C0
:101A6800831264001F3083164D028A150A128312EE
:101A78000318482D8A0199240A308316CD078A1540
:101A88000A128312031C352D8316DC30CB0040303C
:101A9800CC000A30CD00831264001F3083164D023B
:101AA8008A150A1283120318632D8A0148240A3002
:101AB8008316CD078A150A128312031C502D0F3086
:101AC800A300A0308A013C218A01F727C530FB001A
:101AD800FC0183164C30B70083128A150A12DF20E6
:101AE80083164230B60083128A0139228316BA015E
:101AF80083126400133083163A028A150A1283127D
:101B08000318B92D83163A08123C8A150A12831253
:101B1800031CB02D8A150A1297258316B400831268
:101B28008A150A12B02D0D308A0083163A088312DE
:101B38008207203442347934203443344F344D34CE
:101B4800503453347934733428346334293420348A
:101B580032343034303433348A0131228316BA0AAD
:101B68008A150A128312031D7D2D0B30A300B8308D
:101B78008A013C218A01F72783161030DC000430E3
:101B8800DA002030DE006E30DD0083128A01402545
:101B980083166E30DE007830DB0083128A019125CF
:101BA8006430FB00FC0183164C30B70083128A15A1
:101BB8000A12DF2083164230B60083128A013922C6
:101BC8008316BA01831264000A3083163A028A1512
:101BD8000A12831203181A2E83163A08093C8A152A
:101BE8000A128312031C112E8A150A120126831663
:101BF800B40083128A150A12112E0E308A00831639
:101C08003A088312820753345934533454344534D0
:101C18004D3420344C344F3447348A0131228316F2
:101C2800BA0A8A150A128312031DE72DA030FB0099
:101C3800FC0183164F30B70083128A150A12DF2081
:101C480083164230B60083128A0139228316BA01FC
:101C580083126400083083163A028A150A12831226
:101C680003185E2E83163A08073C8A150A12831257
:101C7800031C552E8A150A1247268316B4008312B0
:101C88008A150A12552E0E308A0083163A088312D6
:101C98008207413443345434493456344934543433
:101CA80059348A0131228316BA0A8A150A12831214
:101CB800031D2D2E8130FB00FC0183164F30B70029
:101CC80083128A150A12DF2083164230B600831267
:101CD8008A0139228316BA01831264000A308316F6
:101CE8003A028A150A1283120318A42E83163A0898
:101CF800093C8A150A128312031C9B2E8A150A12A4
:101D08008B268316B40083128A150A129B2E0E3076
:101D18008A0083163A0883128207393438343734F4
:101D280036343534343433343234313430348A014F
:101D380031228316BA0A8A150A128312031D712EDC
:101D4800E330FB000130FC0083164C30B7008312EF
:101D58008A150A12DF2083164230B60083128A01E0
:101D680039228316BA0183126400063083163A02B8
:101D78008A150A1283120318E72E83163A08053CBF
:101D88008A150A128312031CDE2E8A150A12D2261D
:101D98008316B40083128A150A12DE2E0E308A00CA
:101DA80083163A088312820748344F345534523424
:101DB8004C3459348A0131228316BA0A8A150A1218
:101DC8008312031DB82E83161030DC007830DB0038
:101DD8002030DE006E30DD005D08A800A9015C0837
:101DE800A600A7018312831626088312A000831673
:101DF80027088312A10083165B0883128A018A21AF
:101E08008A150A12031D6E2F831622088312A0005A
:101E1800831623088312A1008A011621200883163D
:101E2800A200831221088316A300640080302202D6
:101E38008A150A128312031C2C2F01308316A8025C
:101E48000030031C013EA90283128A150A12312FA1
:101E58008316A80A0319A90A83128316280883126D
:101E6800A000831629088312A10083165D08831237
:101E78008A018E218A150A12031D4B2FFF30831603
:101E88005D07A800FF300318013EA90083128316DE
:101E980028088312A000831629088312A10083163C
:101EA8005E0883128A0186218A150A12031D632F90
:101EB800013083165E07A800A901A90D83128A01C3
:101EC8005E228316A60A0319A70A8A150A12831224
:101ED800031DF72EF030FB00FC0183164C30B700D1
:101EE80083128A150A12DF2083164230B600831245
:101EF8008A0139228316BA01831264000D308316D1
:101F08003A028A150A1283120318B72F83163A0861
:101F18000C3C8A150A128312031CAE2F8A150A126A
:101F28009B278316B40083128A150A12AE2F0F302E
:101F38008A0083163A08831282075434653472344F
:101F48006D3469346E3461346C3420344D346F34FC
:101F5800643465348A0131228316BA0A8A150A1252
:101F68008312031D812F1030FB000130FC00831603
:101F78004C30B70083128A150A12DF2083164230CC
:101F8800B60083128A0139228316BA0183126400CB
:101F98000D3083163A028A110A1683120318012893
:101FA80083163A080C3C8A150A128312031CF82F70
:101FB8008A150A12E5278316B40083128A150A12B5
:101FC800F82F0F308A0083163A0883128207573495
:101FD80061346934743469346E3467342E342E3481
:101FE8002E342E342E342E348A0131228316BA0A26
:101FF8008A150A128312031DCB2F5030FB000130C3
:10200800FC0083164C30B70083128A150A12DF20B1
:1020180083164230B60083128A0139228316BA0128
:10202800831264000E3083163A028A110A1683124C
:1020380003184C2883163A080D3C8A110A16831295
:10204800031C43288A110A162F208316B400831212
:102058008A110A16432810308A0083163A08831218
:102068008207553473346534203447344C3455343E
:10207800543449344C34203431342E3433348A01C6
:1020880031228316BA0A8A110A168312031D1528EB
:102098000730BA004030B8002030AA00AB01AE01CA
:1020A800AF0152308A019B2065308A019B20613044
:1020B8008A019B2064308A019B2079308A019B2009
:1020C8003A308A019B200A308A019B200D308A0110
:1020D8009B200730BA008030B8002030AA00AB013E
:1020E8008A0169205D3C8A110A16031D74288A0139
:1020F80069208316D20052088312A00063308A0137
:102108008121B200831652088312A00043308A014D
:102118008121B400320834048A110A16031D7B2A6F
:10212800831652088312A00073308A018121B200FD
:10213800831652088312A00053308A018121B4000B
:10214800320834048A110A16031D862A8316520897
:102158008312A00071308A018121B20083165208CF
:102168008312A00051308A018121B400320834045E
:102178008A110A16031D912A831652088312A00099
:1021880074308A018121B200831652088312A0009C
:1021980054308A018121B400320834048A110A16A5
:1021A800031D9C2A831652088312A0006C308A01F2
:1021B8008121B200831652088312A0004C308A0194
:1021C8008121B400320834048A110A16031DBD2A7D
:1021D800831652088312A00072308A018121B2004E
:1021E800831652088312A00052308A018121B4005C
:1021F800320834048A110A16031DB22A83165208BB
:102208008312A00062308A018121B200831652082D
:102218008312A00042308A018121B40032083404BC
:102228008A110A16031DA72A831652088312A000D2
:102238006B308A018121B200831652088312A000F4
:102248004B308A018121B400320834048A110A16FD
:10225800031DEB2A831652088312A00064308A01FA
:102268008121B200831652088312A00044308A01EB
:102278008121B400320834048A110A16031DF42A95
:10228800831652088312A00065308A018121B200AA
:10229800831652088312A00045308A018121B400B8
:1022A800320834048A110A16031DF02A83165208CC
:1022B8008312A00070308A018121B200831652086F
:1022C8008312A00050308A018121B40032083404FE
:1022D8008A110A16031D022B831652088312A000C6
:1022E80075308A018121B200831652088312A0003A
:1022F80055308A018121B400320834048A110A1643
:10230800031D152B831652088312A00078308A010A
:102318008121B200831652088312A00058308A0126
:102328008121B400320834048A110A16031DC52A13
:10233800831652088312A00079308A018121B200E5
:10234800831652088312A00059308A018121B400F3
:10235800320834048A110A16031DD82A8316520833
:102368008312A00066308A018121B20083165208C8
:102378008312A00046308A018121B4003208340457
:102388008A110A16031D252B831652088312A000F2
:1023980068308A018121B200831652088312A00096
:1023A80048308A018121B400320834048A110A169F
:1023B800031D352B831652088312A00076308A013C
:1023C8008121B200831652088312A00056308A0178
:1023D8008121B400320834048A110A16031D8A2B9D
:1023E800831652088312A0006D308A018121B20041
:1023F800831652088312A0004D308A018121B4004F
:10240800320834048A110A16031D122D8316520845
:102418008312A0006E308A018121B200831652080F
:102428008312A0004E308A018121B400320834049E
:102438008A110A16031D942C831652088312A000D1
:102448006F308A018121B200831652088312A000DE
:102458004F308A018121B400320834048A110A16E7
:10246800031DEF2B831652088312A00061308A01E6
:102478008121B200831652088312A00041308A01DC
:102488008121B400320834048A110A16031DF52B81
:10249800831652088312A00067308A018121B20096
:1024A800831652088312A00047308A018121B400A4
:1024B800320834048A110A16031DE82B83165208C1
:1024C8008312A00077308A018121B2008316520856
:1024D8008312A00057308A018121B40032083404E5
:1024E8008A110A16031DE12B8A110A164C288A152F
:1024F8000A1243228A150A1222238A0186238A1184
:102508000A164C288A150A1243228A150A1222230F
:102518008A0100248A110A164C288A150A124322B5
:102528008A150A1222238A0199248A110A164C282C
:102538008A150A1243228A150A1222238A0148247C
:102548008A110A164C288A150A12B7228A150A1205
:102558009E228A01E9248A110A164C288A150A1231
:10256800B7228A150A129E228A01F1268A110A16B2
:102578004C288A150A12B7228A01E4258A110A16FC
:102588004C288A150A1243227F088316DC0030087B
:10259800DB003108DE0083128A150A129E228A01A6
:1025A80091258A110A164C288A150A1243227F0897
:1025B8008316DE003008DD003108DC0083128A153E
:1025C8000A129E228A0140258A110A164C288A017D
:1025D800F7278A110A164C2883160130C500831282
:1025E8008A150A12F6218A150A122B238A015E22FD
:1025F8008316C50183128A110A164C2883164C309B
:10260800B70083128A150A12F6218A150A122B239B
:102618008A150A129E228A150A122C218A110A1674
:102628004C288A150A1243228A150A122B2383166C
:102638003108B50083128A150A1263218A110A1615
:102648004C288A150A129E228316C601FF30C7003D
:10265800C9017F30CA0083128A01E9248A110A1647
:102668004C2883164C30B70083128A150A12F621BB
:102678008A150A122B2383164808DF0083128A154D
:102688000A129E22640083163508403C8A110A16F5
:1026980083120319872B6400831635083B3C8A1183
:1026A8000A168312031D622B83162030B50083128D
:1026B8008A150A122C218A110A16692B83163508E5
:1026C800B30083128A150A122C2108308316A60734
:1026D8000318A70A26088312A00083162708831266
:1026E800A100A301EF308A018F218A110A16031D68
:1026F800812B83165F08C80083128A150A129E224E
:102708008A110A16462B8A110A164C2883164D3050
:10271800B70083128A150A12F6218A150A122B238A
:1027280083162608DF002808E00083128A150A129B
:102738009E22640083163508403C8A110A168312CB
:102748000319DE2B6400831635083B3C8A110A16F0
:102758008312031DB92B83162030B50083128A1506
:102768000A122C218A110A16BC2B8A150A122C214E
:1027780083165F08A600A7010830A8070318A90A4E
:1027880028088312A000831629088312A100A30138
:102798007F308A018F218A110A16031DD82B8316D0
:1027A8006008A800A90183128A150A129E228A11BC
:1027B8000A169D2B8A110A164C2883160230B90076
:1027C80083128A110A16F92B83160330B900831273
:1027D8008A110A16F92B8316B90183128A110A166F
:1027E800F92B83160130B90083128A150A12B72211
:1027F800831646088312F600831647088312F500ED
:10280800831649088312F80083164A088312F700D2
:102818007508F3007608F4007308A0007408A10096
:102828007808A30077088A018B218A110A16031DEC
:102838008E2C640083163908003C8A110A1683120C
:10284800031D402C8A150A12B7210730BA00103030
:10285800B8000730BB000830B900A0308A0120203A
:1028680074088A01202073088A0120207F088A01C1
:102878001E200A308A013B21640083163908013C76
:102888008A110A168312031D622C0730BA00103011
:10289800B8000730BB000830B900A0308A012020FA
:1028A80074088A01202073088A0120208A010520E3
:1028B8008316B50083128A150A12A12164008316B3
:1028C8003908023C8A110A168312031D752C8A15D1
:1028D8000A12B721730803178D0003137F088A01B2
:1028E8002D21640083163908033C8A110A168312C5
:1028F800031D872C73088A0125218316B5008312CE
:102908008A150A12A121F30A0319F40A8A110A1670
:10291800031D102C8316B90183128A110A164C283C
:102928008A150A12B72283164908A800A90183123A
:10293800831628088312A000831629088312A10091
:1029480083164A0883128A018A218A110A16031DEE
:102958000F2D83164608A600A701831283162608A2
:102968008312A000831627088312A1008316470844
:1029780083128A018A218A110A16031D062D203026
:10298800A600A701831628088312A2008316290827
:102998008312A3008A01BE21B2002508B300831662
:1029A80026088312A000831627088312A100083086
:1029B800A200A3018A01A221B4002108B5003208AF
:1029C800B40733080318013EB50700303407FB008D
:1029D80010300318013E3507FC008A150A12DF2063
:1029E8008A01432283164408B50083128A150A1205
:1029F800A1218316A60A0319A70A8A110A168312A7
:102A0800031DB22C8316A80A0319A90A8A110A16EB
:102A18008312031D9C2C8A110A164C288A150A1247
:102A2800B72283164908A800A9018312831628082B
:102A38008312A000831629088312A10083164A086E
:102A480083128A018A218A110A16031D5D2D8316B5
:102A58004608A600A7018312831626088312A00041
:102A6800831627088312A1008316470883128A0158
:102A78008A218A110A16031D542D8A150A12B721B4
:102A88007F088316B40083128A150A1263218316FD
:102A9800A60A0319A70A8A110A168312031D302DE4
:102AA8008316A80A0319A90A8A110A168312031D94
:0A2AB8001A2D63008A110A165D2D25
:02400E00753FFC
:00000001FF
